S31508000000280C002061010008870100088901000802
S3150800001000000000000000000000000000000000D2
S315080000200000000000000000000000008B0100082E
S3150800003000000000000000008D0100088F01000884
S31508000040910100089101000891010008910100083A
S31508000050910100089101000891010008910100082A
S31508000060910100089101000891010008910100081A
S31508000070910100089101000891010008910100080A
S3150800008091010008910100089101000891010008FA
S3150800009091010008910100089101000891010008EA
S315080000A091010008910100089101000891010008DA
S315080000B091010008910100089101000800F002F87A
S315080000C000F03EF80CA030C8083824182D18A246AF
S315080000D0671EAB4654465D46AC4201D100F030F887
S315080000E07E460F3E0FCCB6460126334200D0FB1A99
S315080000F0A246AB46334318475C1C00007C1C000034
S31508000100103A02D378C878C1FAD8520701D330C852
S3150800011030C101D504680C60704700000023002434
S3150800012000250026103A01D378C1FBD8520700D320
S3150800013030C100D50B6070471FB51FBD10B510BD87
S3150800014000F0F8F81146FFF7F7FF01F089FD00F017
S3150800015010F903B4FFF7F2FF03BC00F017F900002B
S315080001600F4880F308880F480168090E0E4A914225
S3150800017005D10E480E4901600E480F4901600F4827
S3150800018080470F480047FEE7FEE7FEE7FEE7FEE783
S31508000190FEE700000B480C490C4A0D4B704700005F
S315080001A0280C0020040000001F0000001810024060
S315080001B001000000000001400000000019150008B9
S315080001C0BD00000828060020280C0020280800206A
S315080001D028080020002203098B422CD3030A8B42ED
S315080001E011D300239C464EE003460B433CD4002221
S315080001F043088B4231D303098B421CD3030A8B4233
S3150800020001D394463FE0C3098B4201D3CB01C01A00
S31508000210524183098B4201D38B01C01A52414309CB
S315080002208B4201D34B01C01A524103098B4201D3B9
S315080002300B01C01A5241C3088B4201D3CB00C01A26
S31508000240524183088B4201D38B00C01A524143089E
S315080002508B4201D34B00C01A5241411A00D20146C3
S315080002605241104670475DE0CA0F00D0494203105C
S3150800027000D34042534000229C4603098B422DD3AB
S31508000280030A8B4212D3FC22890112BA030A8B4253
S315080002900CD3890192118B4208D3890192118B42A2
S315080002A004D389013AD0921100E08909C3098B4227
S315080002B001D3CB01C01A524183098B4201D38B016A
S315080002C0C01A524143098B4201D34B01C01A52410D
S315080002D003098B4201D30B01C01A5241C3088B4252
S315080002E001D3CB00C01A524183088B4201D38B003D
S315080002F0C01A5241D9D243088B4201D34B00C01AC7
S315080003005241411A00D20146634652415B101046DB
S3150800031001D34042002B00D54942704763465B1023
S3150800032000D3404201B50020C046C04602BD704712
S3150800033070477047754600F025F8AE4605006946D1
S315080003405346C008C000854618B020B5FFF722FFFF
S3150800035060BC00274908B6460026C0C5C0C5C0C54A
S31508000360C0C5C0C5C0C5C0C5C0C5403D49008D464D
S31508000370704710B50446C046C0462046FFF7E9FE5A
S3150800038010BD000000487047C80500200149182024
S31508000390ABBEFEE726000200704700F088FBFCE7CC
S315080003A010B500F045FB01280ED0084C207801282E
S315080003B00AD101F0E1F86168FF31F531884203D3CB
S315080003C00020207000F094FB10BD0000D80000202B
S315080003D010B5044C0120207001F0CEF86060FFF7DC
S315080003E0DFFF10BDD800002010B500F068FB00F054
S315080003F055FB01F0C9F800F029FF00F009FBFFF7EB
S31508000400E7FF10BD10B500F052FB01F0D7F800F079
S3150800041013FBFFF7C5FF10BD10B501214C0620469A
S3150800042000F03CFF0021204600F038FF10BD000018
S3150800043010B5827A0123194691402A4A14681C434A
S315080004401460D3698B43D361037B002B12D1D36825
S315080004508B43D360C38844881B042343847AE4000F
S31508000460A4182364838804881B042343847AE4003D
S31508000470A4186364037B012B12D1D3680B43D360A2
S31508000480038844881B042343847AE400A41823645D
S315080004908388C4881B042343847AE400A41863640D
S315080004A0C37A002B06D053680B4353600389002B8D
S315080004B004D006E053688B435360F7E753698B43D0
S315080004C053610389012B02D153690B435361407B66
S315080004D0012802D1D0690843D0611068400840005D
S315080004E0106010BD0066004010B5002203680224A3
S315080004F0A34303600368012423430360384B00E0E9
S31508000500521C4468E40701D19A42F9D14268D207DD
S315080005103ED08C798022012C3CD004689443046038
S31508000520CC794022012C39D00468944304600C7AB3
S315080005302022012C36D00468944304604C7A102299
S31508000540012C33D00468944304608C7A0822012C69
S3150800055030D0046894430460CC7A0422012C2DD050
S315080005600468944304608A78CC7892072406224368
S315080005700C79240422434C79098824052243491E10
S315080005800A43C261016849084900016000211AE06E
S31508000590002010BD046814430460C1E704681443CE
S315080005A00460C4E7046814430460C7E70468144396
S315080005B00460CAE7046814430460CDE7046814437A
S315080005C00460D0E7491C4268D20701D09942F9D1A4
S315080005D04068C00701D0002010BD012010BD0000F2
S315080005E0FFFFFF0002460020002905D0012902D19D
S315080005F010698007800F7047D0688007800F7047A2
S3150800060030B50B011B18FF3381331C6B04252C40B6
S315080006101472002C2AD01C6BE40854601C6B02254B
S315080006202C4054725C6B2407240F94725C6B240A6A
S31508000630D4749C6BD4729C6B240A14739C6B240C24
S3150800064054739C6B240E9473DC6BD473DC6B240A92
S315080006501474DC6B240C5474DB6B1B0E937420220D
S31508000660002907D001691143016130BD1C6B640D77
S315080006701460D3E7C1681143C16030BD00218171A0
S31508000680C171017241728172C1728170C170032198
S3150800069001710221417101210180704730B502467E
S315080006A0002093685B010AD49068000101D50120F7
S315080006B005E09068C00001D5022000E00420042867
S315080006C038D003019A18FF3281321368DB07DB0F33
S315080006D013600B7A002B2ED014684D681C434B7A96
S315080006E0ED002B431C4314608B7A1B071B0F8B7280
S315080006F053681B091B01536053688C7A2343536064
S315080007008C7BCB7A240623434C7B0D7B24042D0259
S315080007102C43234393608C7CCB7B240623434C7C5D
S31508000720097C240409020C432343D360116801237E
S315080007301943116030BD13684C7A23430C8864054D
S3150800074023431360D0E700000022002904D00129C2
S3150800075006D002290BD107E082681948024006E054
S3150800076082681848024002E0826817480240174922
S31508000770501A8A421CD007DC002A15D014481018D3
S3150800078014D002280DD117E0FF38FF38023815D0EB
S31508000790104940180ED001214904884201D1012090
S315080007A000E00020C0B270470220FBE70020F9E70E
S315080007B00020F7E70020F5E70120F3E70120F1E73D
S315080007C003000004000300080000031000010008ED
S315080007D0FFFFFFFB0003FFF7F7B58CB0174601A82C
S315080007E000F078FD03980B900024124E6500A919B5
S315080007F0705D497841180C98491C41430B98FFF7DE
S31508000800E9FC00290FD10D9980B208800A49401EDB
S31508000810884208D86000305C3870A819407878702B
S3150800082001200FB0F0BD641CE4B2122CDED3002008
S31508000830F7E700007A1C0008FF03000070B58AB0CD
S31508000840012502951D480068019001AA02A91C48C5
S31508000850FFF7C2FF012803D093211AA0FFF79DFDD9
S31508000860224E3046FFF7D8FD07A8FFF707FF0024FA
S3150800087008AA9470D47009946A469477D477117943
S3150800088008AA491E11706A46507908AA401E507077
S315080008906A461089908307A93046FFF725FE6A46FF
S315080008A09475D47515769481D48114825482948271
S315080008B0557603A8FFF7BCFD0AB070BD781C000882
S315080008C020A107002E2E5C2E2E5C2E2E5C2E2E5C72
S315080008D0536F757263655C41524D434D305F535497
S315080008E04D333246305C63616E2E6300006400400F
S315080008F0F0B585B0054600260024184F0021384675
S31508000900FFF770FE002825D06A4600213846FFF713
S3150800091077FE6846007A1249002803D1009A8A426F
S3150800092000D10124042806D101220198D2071043D8
S31508000930884200D10124012C0CD10021684604E02C
S315080009404218D27A6A54491CC9B26A46927A8A42CD
S31508000950F6D80126304605B0F0BD00000064004018
S315080009606706000030B585B0024600206B4618724F
S315080009700E4B00936B465872997204E0145C1D186E
S31508000980EC72401CC0B28842F8D3094C694620462E
S31508000990FFF784FE054601E000F089F8294620465F
S315080009A0FFF7D2FE0228F7D005B030BDE1070000F8
S315080009B0006400407047000009480078002807D006
S315080009C0012807D0022807D0032807D040207047FF
S315080009D04020704708207047002070470020704765
S315080009E0E000002009480078002807D0012807D031
S315080009F0022807D0032807D04020704740207047B8
S31508000A00082070470020704700207047E00000204B
S31508000A1010B501F079F8FFF711FF044C012020709A
S31508000A2000F058FE0020207010BD0000E0000020F5
S31508000A3010B501F077F810BD10B50A48FFF758FF52
S31508000A40094C012803D12070064801F075F80548BD
S31508000A5000F072FE012804D100202070014801F040
S31508000A606BF810BDF0000020E000002070B50546C8
S31508000A700C46094E3078012803D1E1B22846FFF723
S31508000A8071FF3078002803D1E1B2284600F0A8FEAD
S31508000A9001F0BCF870BD0000E000002010B500F0C1
S31508000AA001F810BD10B5642000F098FB10BD10B514
S31508000AB000F001F810BD10B500F096FB10BD10B59A
S31508000AC000F001F810BD72B6704762B6704770B58F
S31508000AD005460C46164605E020782870641C6D1CF1
S31508000AE0FFF7E5FF3046761EB6B20028F4D170BD92
S31508000AF010B500F0AFFB00281CD000F01DF8002848
S31508000B0018D0FFF757FF00F053FD0121084600F003
S31508000B10D3FB00F097FB01460120C0224007FFF7F0
S31508000B20D6FF032000F0A0FC00F08CFB4468FFF71A
S31508000B30CCFFA04710BD000010B500F047FB01210F
S31508000B404903044800F0CCFA002801D0012010BD62
S31508000B50002010BD000800480149C8607047000021
S31508000B6000200240F0B506460B273F04384600F041
S31508000B706DF804280FD1084C206902252843206106
S31508000B8066612069402108432061384600F05EF816
S31508000B902169A9432161F0BD0020024004200849CB
S31508000BA0CA68D20701D001207047CA68D20601D5A3
S31508000BB002207047C9684907FBD503207047000023
S31508000BC000200240024801698022114301617047F2
S31508000BD000200240F8B505460E46002000900B2777
S31508000BE03F04384600F032F804280ED10E4C20692E
S31508000BF00121084320612E80384600F027F8042892
S31508000C0004D02169490849002161F8BDAD1C009549
S31508000C100098310C0180384600F018F82169490817
S31508000C2049002161F8BD000000200240044801691E
S31508000C30090603D50349416003494160704700002E
S31508000C400020024023016745AB89EFCD00B5034676
S31508000C50FFF7A4FF02E0FFF7A1FF5B1E012801D101
S31508000C60002BF8D1002B00D1052000BDFEB50446A7
S31508000C700D4616461F46680A400200902068401C2A
S31508000C8005D12046009900F00DF900282CD02168DE
S31508000C900098814206D02046009900F015F90446CE
S31508000CA0002C23D02068281A05192D1D0098FF301E
S31508000CB0FF3002300190FFF7FAFE281B0121001FC2
S31508000CC04902884207D32046019900F0FDF80446F8
S31508000CD0002C0DD0251D3078761C28706D1C7F1EC3
S31508000CE0002FE8D10120FEBD0020FEBD0020FEBD7C
S31508000CF00020FEBD10B50C480068401C04D00A4808
S31508000D0000F04CF900280AD008480068401C04D0B6
S31508000D10064800F043F9002803D0012010BD002042
S31508000D2010BD002010BD0000800300207C010020BB
S31508000D3070B504460E46204600F052F80546A0193E
S31508000D40401E00F04DF80146FF2D05D0FF2903D0BF
S31508000D50284600F003F870BD002070BD70B5054642
S31508000D600C46A54201D9002070BD042D01D3122CD2
S31508000D7001D9002070BDFFF759FF3420FFF7ECFEBC
S31508000D80FFF70CFF012812D0284600F047F8054661
S31508000D90204600F043F80646204600F059F8301879
S31508000DA0401E401B401C4001060C002411E0FFF7C2
S31508000DB009FF002070BDFFF77AFEE0024019FFF731
S31508000DC0D1FE042803D0FFF7FDFE002070BD641C89
S31508000DD0A4B2B442EFD3FFF7F5FE012070BD0000C0
S31508000DE070B5054600240C4EFFF761FE21460C201F
S31508000DF041437058A84209D8891949684018A84239
S31508000E0004D90C204443A019007A70BD641CE4B2CE
S31508000E100F2CE9D3FF2070BDA01C000870B506464C
S31508000E2000240A4DFFF743FE0C2060434019007A60
S31508000E30B04203D10C204443285970BD641CE4B267
S31508000E400F2CEFD30020C04370BD0000A01C000883
S31508000E5070B5064600240A4DFFF729FE0C206043AC
S31508000E604019007AB04204D10C2044436019406806
S31508000E7070BD641CE4B20F2CEED3002070BD0000D8
S31508000E80A01C0008004870470020000800200349FD
S31508000E90C043086002490860704700007C010020D2
S31508000EA08003002010B5CA0501D0002010BD0268D5
S31508000EB08A4201D1012010BD02C001225202FFF769
S31508000EC006FE012010BD000070B504460D460E480A
S31508000ED0844201D10D4C0AE00D48854202D10A4CE4
S31508000EE0054604E0204600F059F8002807D02946B0
S31508000EF02046FFF7D7FF002803D0204670BD002004
S31508000F0070BD002070BD0000800300207C01002019
S31508000F10002000080B480168426851188268511879
S31508000F20C2685118026951184269511880694018F7
S31508000F300449C03109680818002801D00020704704
S31508000F40012070470020000870B504460D46164675
S31508000F502046FFF745FFFF2811D06019401EFFF70E
S31508000F603FFFFF280BD0600A40020949884208D192
S31508000F702B46324621460748FFF778FE70BD00200B
S31508000F8070BD2B46324621460348FFF76FFE70BDFB
S31508000F9000200008800300207C010020F8B50546E3
S31508000FA0012000902868FFF71BFFFF2819D0FFF7DC
S31508000FB03DFE3420FFF7D0FDFFF7F0FD012812D0E3
S31508000FC000242868A100461848194768FFF76FFDEE
S31508000FD039463046FFF7FEFD042808D00020009069
S31508000FE00EE00020F8BDFFF7EDFD0020F8BD3068E3
S31508000FF0B84202D00020009002E0641C802CE0D3A6
S31508001000FFF7E0FD0098F8BD08B5002000900E48EF
S315080010100168491C15D0416882685118C268511880
S31508001020026951184269511882695118C0694018F5
S31508001030C043401C00906A4604210448FFF784FF19
S3150800104008BD012008BD000080030020C02000085C
S31508001050F0B500220325012393400C681C409C42EE
S315080010602AD10C79012C01D0022C12D187685400A0
S315080010702E46A640B74387604E79A6408468264325
S31508001080866084889C43848084888B7993401C433B
S315080010908480066853002C469C40A64306600E7959
S315080010A007689E403E430660C668A643C660CC797C
S315080010B09C40C3681C43C460521C102ACBD3F0BDA5
S315080010C010B54B07DB0E9A40C90889000818016A53
S315080010D00F249C40A1430162016A1143016210BDBD
S315080010E002460020128A0A4200D001207047018574
S315080010F07047816170470000FEB501214F043846EC
S3150800110000F0B0F8202000900125684605710024FB
S31508001110847103264671C47109206946C006FFF723
S3150800112097FF09202021C006FFF7E1FF0121C80427
S3150800113000F098F868460471C4716803009069461F
S315080011402048FFF785FF0121384600F099F801216C
S31508001150384600F087F8092001220221C006FFF769
S31508001160AFFF092001220321C006FFF7A9FF0C20C3
S31508001170009068464671022707718471C571092077
S315080011806946C006FFF764FF0121480600F078F8B3
S315080011900121880400F066F8042208210A48FFF7AE
S315080011A08FFF042209210848FFF78AFF30020090C2
S315080011B06846077146718471C57169460248FFF72A
S315080011C047FFFEBD000800480004004810B5092086
S315080011D02021C006FFF78BFF10BD0000014948809B
S315080011E070470000D000002010B500F0C5F90D4C7E
S315080011F0616888420ED321780920C00600290AD0E2
S31508001200002121702021FFF772FF00F0B5F96188EF
S315080012104018606010BD012121702021FFF769FF89
S31508001220F3E70000D000002010B5FFF7EDFE002818
S3150800123002D0FFF75FFD10BD002010BD10B5FFF707
S3150800124077FD10BD10B5FFF71DFE10BD10B5FFF7F1
S315080012501DFE10BD10B5FFF75DFE10BD10B5FFF7FA
S3150800126073FE10BD054A002903D051690143516137
S315080012707047516981435161704700000010024070
S31508001280054A002903D0D1690143D1617047D16964
S315080012908143D1617047000000100240054A0029C9
S315080012A003D01169014311617047116981431161C6
S315080012B07047000000100240054A002903D09169D2
S315080012C001439161704791698143916170470000BC
S315080012D000100240F8B5044600215C4E70680C22E6
S315080012E010405B4D002820D0042820D0082820D0A4
S315080012F00C2839D025607068F02210400009554B3B
S315080013001F5C20680246FA409446626072680727A6
S315080013103F023A40120A9B5C6246DA40A260336B8F
S31508001320DB0524D44C4BE36029E02560E3E7256020
S31508001330E1E771680F208004014070680322D20338
S3150800134010408F0CBF1C00280AD0F06A0107090F4D
S31508001350491C2846FEF73EFF784301462160CAE746
S315080013603E4839464143F9E73D482060C3E773687C
S315080013705B0402D45308E36001E09308E360336B2F
S315080013805F06384B03D4374F1237276100E02361D5
S31508001390376BFF0601D4656100E06061376BBF07F4
S315080013A00ED0376BBF07BF0F012F0BD0376BBF07A8
S315080013B0BF0F022F08D0376BFF43BF0706D006E0E2
S315080013C0A26104E0A06102E0A36100E0A561376BB9
S315080013D0BF03BF0F0FD0376BBF03BF0F012F0CD052
S315080013E0376BBF03BF0F022F09D0376BBF03BF0F81
S315080013F0032F06D006E0E26104E0E06102E0E36163
S3150800140000E0E561376B3F03BF0F0FD0326B120365
S31508001410920F012A0CD0306B0003800F022809D0E6
S31508001420306B0003800F032806D006E0226204E032
S31508001430206202E0236200E02562306B000602D4D7
S3150800144007486062F8BD6162F8BD000000100240FE
S3150800145000127A00C0000020809FD50000093D00D8
S31508001460006CDC0200800000034A116889088900C4
S315080014700143116070470000000001401CB50023BD
S315080014800193009322480168012212041143016066
S3150800149051000524240302680A400092019A521C4E
S315080014A00192009A002A02D1019AA242F3D1016858
S315080014B0890302D50121009100E0009300990129D2
S315080014C025D1144911220A6041684160416841608A
S315080014D041687F22D2039143416041681122120478
S315080014E01143416001680122120611430160016837
S315080014F08901FCD541688908890041604168022252
S315080015001143416041680907890F0229FAD11CBDB8
S31508001510001002400020024010B51448016801225C
S31508001520114301604168124A114041600168114A3D
S3150800153011400160016801229204914301604168EB
S315080015403F22120491434160C16A09090901C16237
S31508001550016BFF22543291430163416B49084900EC
S31508001560416300218160FFF789FF10BD001002402A
S315080015700CB8FF08FFFFF6FE00B500F01FF801489B
S31508001580006800BDE400002000B500F011F8064828
S315080015900449416100218161052202610348016015
S315080015A000BD00007FBB000000E000E0E400002072
S315080015B0014900200861704700E000E0044800691E
S315080015C0C00303D503480168491C01607047000041
S315080015D000E000E0E4000020002904D001680122B0
S315080015E01143016070470168490849000160704766
S315080015F002460020D2690A4200D001207047000046
S3150800160030B58BB004460D4620684008400020607F
S315080016106068032109038843A9680143616020685B
S315080016201E490840EA68696811432A69024311435A
S315080016302160A06803210902884369690143A16002
S3150800164001A8FFF747FE1648844201D107980AE029
S315080016501448844201D1089805E01348844201D110
S31508001660099800E003982168090404D54000296810
S31508001670FEF7B0FD02E02968FEF7ACFD2A685208BD
S315080016808A4200D8401C2168090404D50107490F7D
S31508001690064A10400843A0810BB030BDF3E9FFFFAE
S315080016A0003801400044004000480040F0FF0000B8
S315080016B0826801231B039A43826082680A43826018
S315080016C07047808CC005C00D7047C905C90D0185D6
S315080016D07047000010B586B0E12000020090002097
S315080016E001900290039005900C200490074C6946DF
S315080016F02046FFF785FFA1142046FFF7D9FF0121F1
S315080017002046FFF769FF06B010BD00000044004000
S3150800171070B50446074D20212846FFF769FF0128C2
S3150800172001D0002070BD2846FFF7CBFF20700120AE
S3150800173070BD000000440040F8B50746194C002566
S315080017406078194E00280FD020783018401CFFF713
S31508001750DFFF012817D0FFF70FFF61686431884261
S3150800176000D965700020F8BD0F48FFF7D1FF0128A2
S31508001770F8D130780028F5D0FFF7FEFE60602570B6
S3150800178001206070EEE72078401CC2B222703078E3
S315080017909042E7D1711C3846FFF799F96570012028
S315080017A0F8BD0000E80000208405002070B5054655
S315080017B00A4C80212046FFF71BFF00280BD029463C
S315080017C02046FFF782FF80212046FFF711FF0028F9
S315080017D0F9D0012070BD002070BD00000044004013
S315080017E070B506460D46402D03D97F210EA0FEF79B
S315080017F0D4FD2846FFF7DAFF012803D083210AA083
S31508001800FEF7CBFD00240CE0FFF751F9305DFFF73A
S31508001810CDFF012803D08C2103A0FEF7BEFD641C72
S31508001820A4B2AC42F0D370BD2E2E5C2E2E5C2E2EAA
S315080018305C2E2E5C536F757263655C41524D434D49
S31508001840305F53544D333246305C756172742E6383
S315080018500000000010B5084CFF21E1704168E21D48
S31508001860A06C00F043F9207100206071A071082176
S3150800187020464030818010BD3001002070B500F050
S31508001880CBF90E4C01252570FF20E07000211020B1
S3150800189020716171FFF790F8A071FFF7A3F8E07166
S315080018A0FFF7A0F8000A20726572A5722046082183
S315080018B040308180FFF7CAFC70BD0000300100206F
S315080018C010B5064C0020207000F0A6F9FF20E07045
S315080018D0012120464030818010BD000030010020E3
S315080018E00748FF21C17007498164002101714171D0
S315080018F081710721C01C416008213D3081807047F5
S31508001900300100206E1C00080648FF21C170002126
S315080019100171427842718171C171017206214030AC
S31508001920818070473001002070B50446FFF744F8FF
S315080019306178801E884203DA222000F073F970BDB0
S31508001940104DFF20E87001212846403081806178DB
S3150800195000290AD0A21CA86CFFF780FC00280CD02E
S315080019606178A86C4018A86470BDFFF75DFC002874
S31508001970FAD1312000F056F970BD312000F052F945
S3150800198070BD00003001002010B5094C4168A06CFC
S31508001990FFF754FC002806D0FF20E07001212046FE
S315080019A04030818010BD312000F03CF910BD0000A8
S315080019B03001002070B50546FEF7FEFF0C4C411EAF
S315080019C06A1CA06CFFF74AFC00280CD0FF20E070C8
S315080019D0FEF7F2FFA16C401E4018A06401212046C4
S315080019E04030818070BD312000F01CF970BD0000C8
S315080019F03001002010B5312000F014F910BD0000A8
S31508001A0010B5FFF775F80449FF20C8700248012190
S31508001A104030818010BD00003001002070B5084CB0
S31508001A20FF20E070002525716571FEF7C5FFA071DE
S31508001A30E57125726572072120464030818070BDA8
S31508001A40300100200449FF22CA70406888640248B1
S31508001A5001214030818070473001002070B504466E
S31508001A60FEF7AAFF6178401E884203DA222000F0BA
S31508001A70D9F870BD094D6168A9646278281DFFF719
S31508001A8026F8FF20E8706178A86C4018A86460788A
S31508001A902946401C4031888070BD00003001002076
S31508001AA010B5002000F0BEF810BD000070B5054660
S31508001AB0FEF782FF6A78401E904203DA222000F081
S31508001AC0B1F870BD084C201DA16CFFF700F8FF2087
S31508001AD0E0706978A06C4018A06468782146401CBC
S31508001AE04031888070BD00003001002010B5002309
S31508001AF003E00478401CE318DBB2491E4C1CF8D1FD
S31508001B001360012010BD0000054A00201070906483
S31508001B1011464031C8708880907050707047000038
S31508001B203001002003480078002801D001207047C2
S31508001B30002070473001002070B50178324CFF292B
S31508001B400FD02278012A5ED1F42921D013DCD029BE
S31508001B5036D009DCC92930D0CC293DD0CF293ED191
S31508001B6037E0FFF78BFE3DE0D1292FD0D2292AD0C6
S31508001B70F32934D112E0F5390B0000F064F80A06AF
S31508001B800C303030123015181B30FFF78FFF29E064
S31508001B90FFF764FF26E0FFF755FF23E0FFF75AFE3D
S31508001BA020E0FFF79DFE1DE0FFF77AFF1AE0FFF73A
S31508001BB0ABFE17E0FFF784FE14E0FFF7FBFE11E02B
S31508001BC0FFF7B2FE0EE0FFF729FF0BE0FFF7DCFE9A
S31508001BD008E0FFF715FF05E0FFF70CFF02E02020FD
S31508001BE000F020F8084D4035E878012802D1102089
S31508001BF000F018F80421695E002904DD0120E87068
S31508001C00E01C00F01BF870BD3001002001480021DF
S31508001C10C170704770010020014900204870704764
S31508001C20300100200449FE22CA70087102480221C8
S31508001C3040308180704700003001002010B589B21D
S31508001C40FEF714FF10BD30B47446641E2578641C74
S31508001C50AB4200D21D46635D5B00E31830BC1847F3
S31508001C60FFF74AFAFEF7C0FBFEF7CCFBFCE74F701E
S31508001C70656E424C54000000010105020602060387
S31508001C8007030803090309040A040B040C040C05DA
S31508001C900D050E050F050F061006100710080000A3
S31508001CA000200008000800000400000000280008C2
S31508001CB000080000050000000030000800080000C9
S31508001CC006000000003800080008000007000000B1
S31508001CD0004000080008000008000000004800084E
S31508001CE00008000009000000005000080008000075
S31508001CF00A00000000580008000800000B00000059
S31508001D0000600008000800000C00000000680008D9
S31508001D10000800000D000000007000080008000020
S31508001D200E00000000780008000800000F00000000
S31508001D300080000800800000100000000000010874
S31508001D4000800000110000000080010800800000EB
S31508001D5012000000741D0008C000002030000000BA
S31508001D6000010008A41D0008F0000020380B000040
S31508001D701C0100080000000001020304010203041C
S31508001D800607080900000000000000000000000027
S31508001D900000000004000000000000000000000031
S30908001DA00000000031
S705080000BD35
